S02600002E2E5C62696E5C6F70656E626C745F6F6C696D6578696E6F5F73746D33322E7372656372
S3150800000000500020C51C00080B1D00080D1D000827
S315080000100F1D0008111D0008131D00080000000030
S31508000020000000000000000000000000151D000888
S31508000030171D000800000000191D00081B1D0008F8
S315080000401F1D0008211D0008231D0008251D000886
S31508000050271D0008291D00082B1D00082D1D000856
S315080000602F1D0008311D0008331D0008351D000826
S31508000070371D0008391D00083B1D00083D1D0008F6
S315080000803F1D0008411D0008431D0008451D0008C6
S31508000090471D0008491D00084B1D00084D1D000896
S315080000A04F1D0008511D0008531D0008551D000866
S315080000B0571D0008591D00085B1D00085D1D000836
S315080000C05F1D0008611D0008631D0008651D000806
S315080000D0671D0008691D00086B1D00086D1D0008D6
S315080000E06F1D0008711D0008731D000810B5054C2A
S315080000F0237833B9044B13B10448AFF300800123C6
S31508000100237010BD5C01002000000000F4590008AF
S31508000110084B10B51BB108490848AFF300800848DA
S31508000120036803B910BD074B002BFBD0BDE8104090
S31508000130184700BF0000000060010020F4590008BD
S315080001405C01002000000000154B002B08BF134B74
S315080001509D46A3F5803A00218B460F461348144A5C
S31508000160121A04F03DFF0F4B002B00D098470E4B98
S31508000170002B00D098470020002104000D000D48F0
S31508000180002802D00C48AFF3008004F003FF2000DB
S31508000190290001F0E5FC04F0E9FE00BF00000800B4
S315080001A00050002000000000000000005C01002054
S315080001B044120020000000000000000030B5154C75
S315080001C083B02378054643B1012D4FF48051124878
S315080001D01CD000F069FD03B030BD0121102000F0ED
S315080001E067FD02A94FF4805321F8043D0322142326
S315080001F009488DF807308DF8062000F0E9FC012340
S31508000200012D23704FF480510348E2D100F04EFDD2
S3150800021003B030BDA00300200010014008B501213D
S31508000220034800F03BFD10B100F0A2F8012008BD1C
S3150800023000080140642000F06FB800BF00F072B8F3
S3150800024000B589B000216846202204F0C9FE694637
S31508000250094804F0D1FB50B9009828B19DF8080068
S3150800026080F01000C0F3001009B05DF804FB002010
S3150800027009B05DF804FB00BF0C5000080048704741
S315080002800C50000810B5074C002320460A220649E0
S3150800029084F8243204F02CF810B9012384F82432A7
S315080002A010BD00BF780100202C50000808B508488A
S315080002B090F82432012B04D0BDE80840054804F024
S315080002C0C3BB04F0D1FABDE80840024804F0BCBB41
S315080002D0780100200C500008034890F82432012BBE
S315080002E000D0704704F0C0BA7801002010B5094C58
S315080002F094F82432012B00D010BD214604F052FC9C
S315080003000028F9DA002384F824322046BDE8104094
S3150800031004F0AABA78010020014B1880704700BF84
S31508000320A803002010B502F001F90D4C2368984285
S315080003300ED30C4B1A7862B1002220210A481A7093
S3150800034000F0B4FC02F0F2F8084B1B881844206051
S3150800035010BD0122202104481A7000F0A5FCF1E71F
S31508000360A4030020AA03002000080140A8030020D7
S315080003702021014800F09ABC00080140014608B552
S31508000380064800F0DFFC0121044800F0EFFC0028D5
S31508000390F9D0024800F0D8FCC0B208BD00380040C9
S315080003A010B502F0C3F800F5FA7403E002F0BEF8DF
S315080003B0844206D9FF20FFF7E1FFFF28F6D1012086
S315080003C010BD002010BD00BF10B504210A4800F07A
S315080003D06DFCFF20FFF7D2FFFFF7E2FF10B1012403
S315080003E0204610BD04460421034800F05DFCFF20AA
S315080003F0FFF7C4FF204610BD0014014038B50D466E
S31508000400010604460BD40421224800F04DFCFF20C7
S31508000410FFF7B4FFFFF7D8FF58B9FF2038BD002112
S315080004203720FFF7EBFF012800D938BD04F07F0419
S31508000430E9E744F04000FFF7A1FF280EFFF79EFF0B
S31508000440C5F30740FFF79AFFC5F30720FFF796FFA6
S31508000450E8B2FFF793FF2CB1082C12D18720FFF7DB
S315080004608DFF02E09520FFF789FF0A24FF20FFF79A
S3150800047085FF020604F1FF33D7D513F0FF04F5D143
S3150800048038BD0120FFF77AFF0C2CEED1FF20FFF7CD
S3150800049075FFEAE70014014070B504460D4602F000
S315080004A045F800F1640603E002F040F886421DD9DB
S315080004B0FF20FFF763FFFF28F6D0FE2816D1023487
S315080004C0FF20FFF75BFF04F8020CFF20FFF756FF3B
S315080004D0023D04F8010C04F10204F1D1FF20FFF7F4
S315080004E04DFFFF20FFF74AFF012070BD002070BDB9
S315080004F038B505460C46FFF753FF00B938BD204608
S31508000500FFF73CFFFD2C1ED0AC1C05F2022514F8A3
S31508000510020CFFF733FF023414F8030CFFF72EFF23
S31508000520AC42F4D1FF20FFF729FFFF20FFF726FF93
S31508000530FF20FFF723FF00F01F00A0F10500B0FA27
S3150800054080F0400938BD0120D8E700BF002840F0F8
S31508000550C2802DE9F043AC4D89B02B7803F0020335
S3150800056003F0FF0423B12878C0B209B0BDE8F083D0
S315080005700121202000F09CFB01210820042700F01F
S3150800058097FB01214FF4804000F0A0FB03260DEBFA
S3150800059007014FF010099D48ADF804708DF80790D3
S315080005A08DF8066000F014FB3946984800F07CFB8D
S315080005B04FF4204218230DEB07019548ADF80420A7
S315080005C08DF807308DF8066000F002FB4FF4804284
S315080005D048230DEB07018E48ADF804208DF8073047
S315080005E00DF10C0800F0F4FA4FF482724FF4007320
S315080005F04146ADF80E20ADF8163038220723854857
S31508000600ADF81820ADF81C30ADF80C40ADF8104028
S31508000610ADF81240ADF81440ADF81A4000F064FB8E
S3150800062021467C4800F094FB01217A4800F07CFBC7
S315080006303946764800F038FB4FF4004402A974485E
S31508000640ADF808408DF80A608DF80B9000F0C0FAF6
S3150800065021466F4800F028FB0A2402216D4800F065
S3150800066085FB0028F9D0FF216A4800F06BFB0121C1
S31508000670684800F07BFB0028F9D0013CEDD14FF427
S3150800068000400322182302A9ADF8080060488DF837
S315080006900A208DF80B3000F09BFA04215B4800F025
S315080006A005FB21462046FFF7A9FE0128064614D079
S315080006B0594B0022042155481A6000F0F5FAFF202C
S315080006C0FFF75CFE2B7843F001032B702878C0B245
S315080006D009B0BDE8F0830120704701F027FF4FF409
S315080006E0D57100F57A770820FFF788FE012835D1FD
S315080006F002AC2646FF20FFF741FE06F8010BB0457F
S31508000700F8D19DF80A30012BD2D19DF80B30AA2BCF
S31508000710CED102E0FFF772FE38B101F007FF87423B
S315080007204FF080414FF0A900F4D801F0FFFE874250
S31508000730BED900213A20FFF761FE0028B8D1FF2074
S31508000740FFF71CFE04F8010BA045F8D19DF8083008
S3150800075013F0400F14BF0C2604261EE02146A920DC
S31508000760FFF74CFE01289ABF0226A924344603E067
S315080007702046FFF743FE28B101F0D8FE87424FF026
S315080007800001F5D801F0D2FE874291D94FF40071E5
S315080007901020FFF733FE00288AD11F4B04211B487F
S315080007A01E6000F081FAFF20FFF7E8FD00210C46E5
S315080007B02B78184803F0FE032B704FF4827700F06D
S315080007C0B3FA4FF400760822072341461148ADF8DC
S315080007D01820ADF81C30ADF80C40ADF81040ADF857
S315080007E01240ADF81440ADF81A40ADF80E70ADF8E9
S315080007F0166000F079FA2146064800F0A9FA0121A8
S31508000800044800F091FAAEE600000020001401400A
S31508000810000C014000380040AC03002018B9034B17
S315080008201878C0B270470120704700BF000000204A
S3150800083030B583B018B10424204603B030BD002B70
S31508000840F9D00D4621490978C80701D50324F3E7ED
S315080008501F4901930968090758BF5202012B11461F
S3150800086022D01220FFF7CAFD019B58B101240421AA
S31508000870184800F019FAFF20FFF780FDDCE714F0AE
S31508000880FF0318D028464FF400710193FFF704FEC2
S31508000890019B05F500755C1E0028F0D10124002196
S315080008A00C20FFF7ABFDE2E71120FFF7A7FD019B40
S315080008B018B11C46DBE71C46F1E728464FF40071E1
S315080008C0FFF7EAFDB0FA80F46409D0E700000020DB
S315080008D0AC0300200014014010B582B018B10424FE
S315080008E0204602B010BD002BF9D00C462B490878DB
S315080008F0C00701D50324F3E70978490701D502247F
S31508000900EEE727490968080758BF5202012B37D076
S3150800091011F0060F2BD1114619200093FFF76EFD33
S31508000920009B58B1012404211E4800F0BDF9FF20A0
S31508000930FFF724FDD4E712F0FF030AD02046FC2176
S315080009400093FFF7D5FD009B04F500745A1E002896
S31508000950F1D10093FFF724FD009B0028E2D01C1C70
S315080009604FF0FD0018BF0124FFF708FDDBE7194625
S31508000970972001920093FFF741FD019A009BCAE771
S3150800098011461820FFF73AFD0028CBD12046FE2154
S31508000990FFF7AEFDB0FA80F46409C4E70000002052
S315080009A0AC0300200014014008B104207047834BB3
S315080009B01B78D80701D50320704770B5154684B053
S315080009C00E2900F2A380DFE801F05F65A129A1A145
S315080009D0A1A1A1A15A4C99180800794B1B685B077D
S315080009E000F1B98001240421764800F05DF9FF2062
S315080009F0FFF7C4FC204604B070BD00213A20FFF77B
S31508000A00FDFC0028EED16C1E0335FF20FFF7B6FC6F
S31508000A1004F8010FAC42F8D10024E4E7684E3368C5
S31508000A2013F0040174D000218D20FFF7E7FC00289D
S31508000A30D8D1FF20FFF7A2FC10216846FFF72CFD4E
S31508000A400028CFD03024FF20FFF798FC601E10F056
S31508000A50FF04F8D19DF80A201023120993402B6051
S31508000A60C1E700210920FFF7C9FC0028BAD12846AA
S31508000A701021FFF711FDB0FA80F46409B3E7504B73
S31508000A8000241B681370AEE7FFF79EFCB0FA80F4EB
S31508000A906409A8E700210920FFF7B0FC04460028EE
S31508000AA0A0D110216846FFF7F7FC00289AD09DF8D8
S31508000AB000309B09012B60D09DF805309DF80A602F
S31508000AC09DF8092003F00F019DF807009DF80630F0
S31508000AD001EBD61152009DF80860023102F00602B9
S31508000AE080009B020A4403F4406300EB9611D2B2DD
S31508000AF00B44093A013393402B6074E700210A201E
S31508000B00FFF77CFC00287FF46DAFB0E704246AE7A2
S31508000B100920FFF773FC044600287FF463AF102111
S31508000B206846FFF7B9FC00283FF45CAF336813F05A
S31508000B30020332D09DF80A309DF80B105B009DF831
S31508000B400D2003F07E0303EBD11392090133013A1A
S31508000B5093402B6047E700218D20FFF74FFC0028C4
S31508000B607FF440AFFF20FFF709FC28464021FFF736
S31508000B7093FCB0FA80F4640935E79DF807309DF8D0
S31508000B8008101B049DF8092003F47C13013302EBBB
S31508000B90012213449B022B6025E79DF80B409DF824
S31508000BA00A20E00000F01800C2F3840100EB54109C
S31508000BB04A1C00FB02221C462A6014E7000000209B
S31508000BC0AC03002000140140004870470000AA4208
S31508000BD0CB782DE9F04103F00F06DB0648BF8B788A
S31508000BE00C8848BF1E4314F0FF0F26D00568002363
S31508000BF001274FF00F0803E00133082B1BD00C88A0
S31508000C0007FA03F232EA0404F6D19C0091F803E0ED
S31508000C1008FA04FC25EA0C0506FA04F4BEF1280FC6
S31508000C2045EA040538D0BEF1480F03F1010308BFB1
S31508000C300261082BE3D105600C88FF2C2AD9456888
S31508000C40002301274FF00F0C03E00133082B20D0B7
S31508000C500C8803F1080207FA02F232EA0404F4D116
S31508000C6091F803E09C00BEF1280F04BF426191F899
S31508000C7003E00CFA04F8BEF1480F03F1010325EA74
S31508000C80080506FA04F408BF0261082B45EA0405BC
S31508000C90DED14560BDE8F0814261ADE7836819425F
S31508000CA014BF0120002070470161704741617047F9
S31508000CB029B9054A936923EA000090617047024BF7
S31508000CC09A691043986170470010024029B9054A8D
S31508000CD0D36923EA0000D0617047024BDA691043F2
S31508000CE0D8617047001002404A8830B40C888B8857
S31508000CF02243CC881A430B8922434C898D891A438F
S31508000D0022430388CC892A43224303F441531343DD
S31508000D109BB20380838B30BC23F400631B041B0C3B
S31508000D2083830B8A03827047038829B923F040031B
S31508000D301B041B0C038070479BB243F040030380DF
S31508000D40704700BF81817047808980B2704700BFB5
S31508000D50038829B923F400531B041B0C038070472E
S31508000D609BB243F400530380704700BF03891942BE
S31508000D7014BF01200020704708B538B1064B1B6820
S31508000D801B689847054B18680A3008BD034B0122B3
S31508000D901B681A8208BD00BF3412002038120020D2
S31508000DA008B538B1064B1B689B689847054B186809
S31508000DB00C3008BD034B01221B681A8208BD00BF10
S31508000DC0341200203812002008B51F4B002832D0F4
S31508000DD01E481A6800210180137813F07F0316D085
S31508000DE0012B27D0022B24D1527902F00F039B0046
S31508000DF003F1804303F5B84312061B681FD403F4B6
S31508000E004053B3F5805F0ED1012303700BE0527A8D
S31508000E10930654BF0378022351064CBF43F00103DF
S31508000E2023F0010303700A4B1B681B6998470748A0
S31508000E3008BD084608BD1B6802221A8208BD03F0D1
S31508000E403003102BEFD1DFE73812002008120020FC
S31508000E50341200202DE9F041244F3C68258A2DB92B
S31508000E60267A042E2AD0A38A042603E0A38A9D4262
S31508000E70FAD902269D4228BF1D46A36928469847E7
S31508000E808046002000F01EFE2A460146404600F035
S31508000E90EBFC2946002000F0B3FD638A228A144938
S31508000EA0521B1D44134B2282658230204FF4405258
S31508000EB03C6808801A802672BDE8F0810E4B1A78C5
S31508000EC0012A06D00A4B102207261A802672BDE888
S31508000ED0F0810A490A4A0968054889B20A44520053
S31508000EE0156030223C681D700280E4E73812002045
S31508000EF0401200203E120020B0030020505C004043
S31508000F00023000200B4B0C4A1B685178DA78914264
S31508000F1001D20220704799780029FAD110B59C8829
S31508000F200CB1022010BD05499A720B685B68984798
S31508000F30204610BD38120020EC0000203412002094
S31508000F4038B5104A104C12682368D97858799369CD
S31508000F50984723689A7A0AB9022038BD0028FBD137
S31508000F601A79002AF8D19D78002DF5D1074B1B6810
S31508000F70DB689847236828465979DA78D9721A734C
S31508000F8038BD00BF1012002038120020341200208D
S31508000F9038B5314B1B68187810F07F0003D002284B
S31508000FA006D0022038BD5A7A22F020025A7238BD7D
S31508000FB05A88002AF6D11A79002AF3D15A7922F0EA
S31508000FC080008400150604F18041244D01F5B841DE
S31508000FD009682D784CBF01F0300101F44051A84250
S31508000FE0DFD20029DDD09B7A002BDAD004F18044C9
S31508000FF004F5B8441206236809D503F03003102B0C
S315080010001ED0174B1B685B699847002038BD03F450
S315080010104053B3F5805FF4D1D8B9124B93F82C102E
S3150800102000F0FCFC236823F4804323F070039BB292
S3150800103083F4405343F4004343F080032360E0E71E
S31508001040C4B2204600F0CAFC2046302100F046FC17
S31508001050D7E700F0B1FCE5E738120020EC000020E5
S31508001060341200206000002038B5224B18684279F7
S3150800107022F080018C00150604F180431E4D03F50D
S31508001080B8431B682D784CBF03F0300303F4405374
S31508001090A94201D3022038BD41880029FAD1002B84
S315080010A0F8D0837A002BF5D004F1804404F5B844CF
S315080010B01206236811D523F4E04323F040039BB2BC
S315080010C083F0100343F4004343F0800323600B4B83
S315080010D01B689B699847002038BD23F4804323F09A
S315080010E070039BB283F4805343F4004343F08003B8
S315080010F02360ECE738120020EC00002034120020B0
S31508001100054B1B685A8A10B10868104470478988CD
S315080011108A1A1A82704700BF3812002010B50C4B85
S31508001120002093F82C1000F079FC0A4B1B68187AFB
S31508001130082806D10849094B4FF4805410220C8020
S315080011401A80A0F10900B0FA80F0400910BD00BF6E
S3150800115060000020381200203E12002040120020B5
S3150800116070B5A24DA24A2B6811681A7A82B0092A6C
S315080011703ED0A04A89B20A4452001488640004F199
S31508001180804404F5C04422781A702B6862785A7035
S31508001190A0882E6800F0BAFC708020892E6800F0BE
S315080011A0B5FCB080A2892B680121DA80197222B3B6
S315080011B05878062800F0848000283AD159880029F2
S315080011C000F098808C4C23681B699847032800F028
S315080011D0EA804FF6FF722C68238A934200F08480D7
S315080011E0022836D108232372FFF798FF02B070BD94
S315080011F0DA8801211972002ADAD11A785C7812F095
S315080012007F0236D0012A00F0BF80022A00F0E18072
S31508001210794B20461B685B699847032800F0C38012
S3150800122000283ED02B6808221A72FFF777FF02B013
S3150800123070BD082870D11A785206C3D16F4A0020AB
S315080012409A61588290474FF6FF722C68238A934218
S315080012504AD0002BC6D094F90020002A7FDB684AC2
S315080012604FF44051032311802372FFF757FF02B052
S3150800127070BD092C00F0E180052C00F09B80032C42
S3150800128000F0CA80012CC3D1DA78012AC0D19A8825
S31508001290002ABDD15B7A9B06BAD5FFF779FE0028EE
S315080012A0B6D1534A574B1268002192B213445B00D9
S315080012B01960554A30212B68118006221A72B4E744
S315080012C01A7856067FF47EAF9A784B4C012A00F0BE
S315080012D0BA80022A6BD0032A7FF475AF2268526A55
S315080012E0002AACD106206EE709232372FFF716FF02
S315080012F002B070BD5A6822F47F42B2F5003F7FF40F
S3150800130061AF187810F07F0040F0A0809A88002A14
S315080013107FF458AF3D4A92E70A287FF453AF1A780C
S3150800132002F07F02012A7FF44DAF9A7A002A3FF431
S3150800133049AF598800297FF445AF5A682E4C22F4E4
S315080013407F42B2F5803F7FF43EAF226858799369B1
S3150800135098472B68002840F0B6802D4A6FE7E28848
S31508001360019201998B4217D8934276D2224A126883
S3150800137092F82C108AB2934274D2264B0021197027
S31508001380A282FFF767FD70E70B2C7FF441AFFFF7EA
S31508001390D7FD002885D03BE7174B019A1B682282A8
S315080013A093F82C20ECE72B6809221A723DE722688D
S315080013B0126A95E793F90320002A07DB9A782AB977
S315080013C09A881AB99A7A002A3FF46BAF08221A72D9
S315080013D02BE7012C3FF461AF032C7FF419AFFFF71D
S315080013E043FE00283FF45DAF12E700BF3812002025
S315080013F0505C00400430002010120020790D0008CF
S315080014003E1200200230002040120020C90D0008BC
S31508001410A10D0008B0030020DA78012A7FF4F8AE9F
S315080014209A88002A7FF4F4AE5A7A284942F02002B4
S3150800143009685A72CB69984733E7FFF763FD0028B6
S315080014403FF42FAFE4E62268D26949E701282FD096
S31508001450022811D008461E4CB5E61D4B1B6893F8AA
S315080014602C208DE793FBF1F001FB1033002B87D17D
S31508001470184B0121197083E7587900F00F018A008B
S31508001480040602F18042144C02F5B8421268247828
S315080014904CBF02F0300202F44052A14206D210F0CC
S315080014A0700003D1002A7FF435AF8BE6002089E669
S315080014B0074C58792268936998472B6818B99A7A1D
S315080014C0002A7FF427AF58787DE600BF3412002043
S315080014D010120020B0030020EC000020F8B5304DB3
S315080014E02C68237A022B07D0042B05D0032B09D0AE
S315080014F0052B07D0072B33D008232372BDE8F84005
S31508001500FFF70CBEA369228AB3B1B2B1A68A964286
S3150800151028BF164630469847228A638A921B334468
S31508001520074622826382002000F0DCFA3246014632
S31508001530384600F0ADF9228ACAB9A38A33B31949E5
S315080015402A68194B062010721A68184B92B213446F
S315080015505B0000221A602C683022237A0A80CCE7C6
S31508001560134B1B68DB6898472C680823C5E7114BA3
S3150800157000214FF4405208461A8000F041FA238AA7
S31508001580A28A084930209A42088003D82C68032387
S315080015902372B2E7002BD3D02C6805232372ACE75D
S315080015A03812002040120020505C00400230002013
S315080015B0101200203E120020F8B5234C23681A7A30
S315080015C0022A17D0042A15D0062A05D008221A722C
S315080015D0BDE8F840FFF7A2BD5A78052A13D01B4B81
S315080015E01B689B689847236808221A72BDE8F8406A
S315080015F0FFF794BDFFF72EFC23681A7A1A72BDE826
S31508001600F840FFF78BBD1A7812F07F02E7D1104930
S31508001610DF780E7876B10F4840F60F73056842F406
S3150800162000412B4041F0800101320B43964240F8BD
S31508001630043BF1D1084A47F08007084B17601B683E
S315080016401B6A9847CBE700BF38120020101200200B
S31508001650EC000020005C00404C5C00403412002086
S3150800166070B40C4B1E787EB10B4C002240F60F73FB
S31508001670256842F400412B4041F0800101320B43BA
S31508001680964244F8043BF1D1044B40F080001860C0
S3150800169070BC7047EC000020005C00404C5C0040C9
S315080016A0704700BF70B4074A07490848084E094CF6
S315080016B0094B022515720860236032601B6870BCEE
S315080016C0184700BF1812002034120020900000208E
S315080016D03812002010120020600000202DE9F04F7B
S315080016E0DFF878A1DFF878915746C84685B0002319
S315080016F0DFF870B1544DADF80E30DBF80030534CBE
S3150800170099B21B04524E504AAAF8001040F1908034
S315080017103B8803F00F03990001F1804101F5B841B8
S3150800172089F80030002B2FD14BF6BF73216889B298
S315080017302980298801F030013180298801F4405137
S31508001740298021680B4083F4005383F0200343F477
S31508001750004343F0800323603B88D90641D52368BC
S315080017609BB2ADF80E30BDF80E301B0563D4BDF83C
S315080017700E301804C1D540F68F73019221680B40CC
S315080017802360FFF7ABFE34E00B689BB2ADF80E3072
S31508001790BDF80E30180417D4BDF80E301A06ACD5AD
S315080017A048F60F7299F800302A499B0003F18043E6
S315080017B003F5B843186802401A6099F80030013BEF
S315080017C051F82330984798E740F68F730868224AFD
S315080017D003400B6098F80030013B52F823309847D5
S315080017E0DAE748F60F73019221680B402360FFF78A
S315080017F0E3FE4BF6BF73019A2068118812880340EE
S31508001800C90448BF83F480539704328848BF83F4D9
S315080018100053D506328848BF83F01003940648BFA4
S3150800182083F0200343F40043084A43F0800313601F
S3150800183005B0BDE8F08F40F68F73019221680B4022
S315080018402360FFF78DFCD4E73E120020005C0040C1
S3150800185040120020200000203C00002042120020F8
S3150800186014120020445C0040013252100ED010B40D
S3150800187001F1005101F540514900002330F8024BAF
S3150800188021F8234001339A42F8D110BC704700BFB3
S3150800189001F10051013201F5405152104FEA410160
S315080018A005D051F8043B013A20F8023BF9D17047BC
S315080018B04FF6F873014A034013607047505C0040C6
S315080018C0800000F1804000F5B840036823F4EC433B
S315080018D023F07003194389B201607047800000F154
S315080018E0804000F5B8400368CA0623F4E04323F0B5
S315080018F040039BB248BF83F010038A0648BF83F0B3
S31508001900200343F4004343F080030360704700BF9D
S31508001910800000F1804000F5B8400368CA0423F44B
S31508001920804323F070039BB248BF83F480538A0434
S3150800193048BF83F4005343F4004343F08003036035
S31508001940704700BF800000F1804000F5B84003688A
S3150800195023F4E04323F040039BB283F0300343F4BF
S31508001960004343F080030360704700BF800000F126
S31508001970804000F5B840036823F4804323F07003E1
S315080019809BB283F4405343F4004343F0800303605F
S31508001990704700BF40F60F62800000F1804000F5F6
S315080019A0B8400368134043F4004343F080030360E0
S315080019B0704700BFFFF7EEBF800000F1804000F5DA
S315080019C0B84003685B0408D540F60F7302681340F5
S315080019D043F4404343F0800303607047800000F1FE
S315080019E0804000F5B84003685B0608D540F60F73DB
S315080019F00268134043F4004343F0C0030360704792
S31508001A00044A054B126892B202EBC00003445B001D
S31508001A1019607047505C0040023000200E4A0F4B98
S31508001A2012683E2992B202EBC00003444FEA430310
S31508001A300AD94A09C80604BF02F1FF3292B29202D5
S31508001A4042F400421A6070474A08C90748BF013283
S31508001A5092021A60704700BF505C004006300020B2
S31508001A60064B49081B6849009BB203EBC00000F10E
S31508001A70005000F54050400001607047505C00403F
S31508001A80FFF7EEBF054A064B1268490892B202EB09
S31508001A90C000034449005B0019607047505C004071
S31508001AA004300020FFF7EEBF054B1B689BB203EB23
S31508001AB0C00000F1005000F5405040000088704713
S31508001AC0505C0040FFF7F0BF044A054B126892B21B
S31508001AD002EBC00003445B0018887047505C004066
S31508001AE004300020FFF7F0BF054A064B126892B291
S31508001AF002EBC00003445B001868C0F30900704796
S31508001B00505C004006300020FFF7EEBFC3B2000A63
S31508001B1040EA0320704700BF10B40549054C064A41
S31508001B2000204FF4064320600B80136010BC7047FA
S31508001B303C120020445C0040405C004070B500F058
S31508001B407F0528460E46FFF7DFFF04462846FFF7BF
S31508001B50C9FF224601463046FFF79AFE204670BD69
S31508001B6000B5534B002285B0019202921968514A7A
S31508001B7041F0010119605D684FF41F012A405A605F
S31508001B801A6840F2DC5422F0847222F480321A6019
S31508001B901A68184622F480221A605A6822F4FE024D
S31508001BA05A6099601A6842F480321A6002E0019B12
S31508001BB0A34209D0036803F400330293019B01335F
S31508001BC00193029B002BF2D0394B1B6899036AD507
S31508001BD0394A374B1068194640F0100010601068F3
S31508001BE020F003001060106840F0020010605A6888
S31508001BF05A605A6842F400525A605A6842F480623F
S31508001C005A605A6822F47C125A605A6842F4E812FA
S31508001C105A601A6842F080721A600A68244B920168
S31508001C20FBD519465A6822F003025A605A6842F0F0
S31508001C3002025A604A681E4B02F00C02082AF9D1C1
S31508001C4001210D465A6804AC22F480025A60DA690A
S31508001C50042042F40002DA61FFF72AF824F8045D4A
S31508001C6048232146032615488DF80F308DF80E6057
S31508001C70FEF7AEFF29460420FFF71AF820251023A1
S31508001C8021460E488DF80F308DF80E60ADF80C50D1
S31508001C90FEF79EFF29460948FFF708F800F026FEDA
S31508001CA000F036FEFCE76F21054800F0E7FD8FE7F8
S31508001CB0001002400000FFF8002002400008014022
S31508001CC03C50000806498D460649074A074B9A4282
S31508001CD0BEBF51F8040B42F8040BF8E70448004766
S31508001CE000500020005A0008000000205C01002077
S31508001CF0490100081F49204A002301E041F8043B36
S31508001D009142FBD3FFF72CFFFEE7FEE7FEE7FEE76F
S31508001D10FEE7FEE7FEE7FEE7FEE7FEE7FEE7FEE78D
S31508001D20FEE7FEE7FEE7FEE7FEE7FEE7FEE7FEE77D
S31508001D30FEE7FEE7FEE7FEE7FEE7FEE7FEE7FEE76D
S31508001D40FEE7FEE7FEE7FEE7FEE7FEE7FEE7FEE75D
S31508001D50FEE7FEE7FEE7FEE7FEE7FEE7FEE7FEE74D
S31508001D60FEE7FEE7FEE7FEE7FEE7FEE7FEE7FEE73D
S31508001D70FEE7FEE75C0100204412002000F0F2BCFA
S31508001D8000F036BD034B1B68052B00D0704700F0EA
S31508001D90E9BC00BFB403002070B51749174C0B689F
S31508001DA0174D9BB2238022882B881A40920517D498
S31508001DB0228802F4004213420ED1228802F480627D
S31508001DC0134200D170BD4FF6FF310B4A0D4B11601F
S31508001DD05B68BDE870401847FFF780FC2B88ECE786
S31508001DE04FF6FF53084A0B6013780133DBB21370C2
S31508001DF0FFF7C8FF2B88DBE7445C0040421200204F
S31508001E003C12002060000020B1030020034B9B7A9F
S31508001E1013B1034B05221A60704700BF1812002041
S31508001E20B4030020014B04221A607047B403002053
S31508001E30704700BF062801D0022070470B4B1B686D
S31508001E401A7802F07F02012AF6D110B55C7954B9E6
S31508001E509A78212A07D1064A5C829A61204600F0C0
S31508001E6097F8204610BD022010BD00BF381200208A
S31508001E70911F00080220704709B102207047002808
S31508001E8014BF02200020704710B500F0D7FC054BA0
S31508001E9000241B689C7200F083F8FFF73DFE024B96
S31508001EA01C6010BD38120020B403002010B5264B64
S31508001EB0264A1B68D27900245A729C72DC72204624
S31508001EC0FFF7F6FC20464FF40071FFF7F9FC2046B1
S31508001ED01021FFF703FD20464021FFF7E3FD80218F
S31508001EE02046FFF7CDFD2046FFF764FD184B204638
S31508001EF093F82C10FFF792FD2046FFF737FD214691
S31508001F000120FFF7DDFC4FF480710120FFF7B8FDD3
S31508001F10C0210120FFF7C6FD40210120FFF770FD13
S31508001F2040210120FFF77AFD4FF440510120FFF7C9
S31508001F30EFFC20210120FFF7D1FC2046FFF790FB9C
S31508001F40044B01221A6010BD381200208850000880
S31508001F5060000020B40300200149FFF7D1B800BF94
S31508001F60BC0000200149FFF7CBB800BF580000208D
S31508001F70054B1B68DB78052B04D8044901EBC30124
S31508001F80FFF7BEB80020704738120020C4000020B2
S31508001F900149FFF7B5B800BFB4000020704700BF7D
S31508001FA038B50120FEF70AF9064D074B074C002203
S31508001FB04FF4E051012018601A602A6021801960E8
S31508001FC0104638BD445C0040405C00403C1200208E
S31508001FD000F06CBA10B500F073FA00B910BDFEF740
S31508001FE01DF90028FAD000F0C1FC00F08BFA00F0C9
S31508001FF069FA074B20F0604020F07F00186000F077
S3150800200061FA446800F054FA2346BDE810401847C0
S3150800201008ED00E072B170B50D46561EB6B206441C
S31508002020441E15F8013B04F8013F00F0C7FCB44212
S31508002030F7D170BD704700BF2DE9F041DFF83C804D
S31508002040074646460C4D002401E056F80C5F00F0A2
S31508002050B5FCBD4203D873681D44AF4205D30134AD
S315080020600D2CF2D1FF20BDE8F08104EB440408EB07
S315080020708404207ABDE8F08100600008F05000086A
S315080020802DE9F04107460068FFF7D6FFFF2845D03F
S31508002090244A25482549342350605160D360D368C3
S315080020A013F0010327D11446116941F001011161AA
S315080020B003F1040857F808603D68B2B25A53E2685B
S315080020C01D44D00704D500F079FCE368DA07FAD492
S315080020D0330C6B80E368D90704D500F06FFCE3681E
S315080020E0DB07FAD42B689E420CD1B8F5007F43462D
S315080020F0DED1012007E01369002043F08003136155
S31508002100BDE8F0810020074B1A6922F001021A6126
S315080021101A6942F080021A61BDE8F0810020BDE824
S31508002120F08100BF0020024023016745AB89EFCD4F
S3150800213038B5104B0D46984219D00F4A914208D02F
S315080021400446FFF79DFF10B1C5F3080313B100203D
S3150800215038BD1C462368AB4207D02046294640F8BE
S31508002160045B4FF40072FFF755FF204638BD034C59
S31508002170EAE700BFB803002000600008BC0500209D
S315080021802DE9F8430C46016824F4FF781D464B1CDC
S315080021900746164628F0010832D0884506D0384644
S315080021A04146FFF7C5FF074638B30168641A3C4441
S315080021B0043408F5007807F1040905E016F8013B30
S315080021C0013D04F8013B15D000F0F8FBC9EB040308
S315080021D0B3F5007FF2D338464146FFF7A9FF074615
S315080021E000F1040948B14C4616F8013B013D04F8D4
S315080021F0013BE9D10120BDE8F8830020BDE8F8835A
S31508002200814649F8048B414648464FF40072FFF769
S3150800221001FF3968C1E700BF0349044A4FF0FF339D
S315080022200B601360704700BFBC050020B803002090
S3150800223070B50D4616460446FFF7FEFEFF2814D075
S31508002240681E2044FFF7F8FEFF280ED00A4A24F439
S31508002250FF7323F00103934221462B46324606D0EC
S31508002260BDE870400548FFF78BBF002070BD0448E5
S31508002270BDE87040FFF784BF00600008BC05002079
S31508002280B80300202DE9F0470C460646FFF7D4FEB2
S315080022900546601E3044FFF7CFFE85426BD8EB1E1D
S315080022A0DBB2FB2B67D80F28044664D8464A474852
S315080022B04749342350605160D360D36813F0010650
S315080022C068D11369434F43F00203B846B946136110
S315080022D04FF0030A01E099F808A000F06FFB554596
S315080022E009F10C095DD001360D2EF4D14FF0FF36F9
S315080022F0DFF8E09000254FF0030A01E099F808A0FE
S3150800230000F05CFB544509F10C0957D001350D2D39
S31508002310F4D14FF0FF3900254FF0030A01E097F892
S3150800232008A000F04BFB544507F10C073FD00135D8
S315080023300D2DF4D10023C6EB09094B44C3F38F23B3
S31508002340E3B15F1EBFB206F580651F4C05EB872714
S315080023506661236943F040032361E368DA0704D51D
S3150800236000F02CFBE368DB07FAD4AF422E4605D013
S3150800237005F58065ECE70020BDE8F087124B0120E3
S315080023801A6922F002021A611A6942F080021A6179
S31508002390BDE8F0871369002043F080031361BDE8A8
S315080023A0F087F6B206EB460658F82660A0E7EDB2C7
S315080023B005EB450508EB85056B68BCE7EDB205EB53
S315080023C0450558F82590A6E70020024023016745F1
S315080023D0AB89EFCDF05000080F4B1A68013218D0C0
S315080023E030B599685C68DD6818690C442C445969ED
S315080023F0044498690C44D969231883B00B4402AA8B
S315080024005B4242F8043D04210448FFF711FF03B07C
S3150800241030BD0120704700BFB8030020EC600008FB
S3150800242010B40E490E4B0F4A08681B680E4C12680A
S315080024300C31034409680D48134422680B440168AB
S315080024401344A2680B44D0F8D8101344CB4200F1C9
S31508002450D80010BC0CBF012000207047006000089F
S31508002460046000080860000810600008146000088E
S3150800247008B50A480368013302D0FFF701FE58B1D0
S3150800248007480368013305D0FFF7FAFD003018BF87
S31508002490012008BD012008BD08BD00BFB803002003
S315080024A0BC050020004870470060000872B67047F7
S315080024B062B67047FFF7B0BEFFF7BABEFFF7E2BED7
S315080024C0FFF7AEBFFFF7EEBF08B5FFF785FF00B908
S315080024D008BDBDE80840FFF7CBBF00BF10B4064BE8
S315080024E0064C0749002205201A605C609A6018604D
S315080024F00A6010BC704700BF10E000E03F190100F9
S31508002500C0070020014B00221A60704710E000E067
S31508002510044B1B68DB0303D5034A136801331360B6
S31508002520704700BF10E000E0C0070020044B1B689E
S3150800253013F4803F034B18681CBF013018607047BE
S3150800254010E000E0C0070020B2B1002370B41E46B8
S31508002550541EE4B201346400020F092A02F1300560
S3150800256086BF3732CA54CD54CA180233A3424FEA3B
S3150800257000105670F0D170BC704700BF012838B5FE
S3150800258004460D4604D94FF4FC710F4800F076F95D
S3150800259004EB44040D48E4000319597C1A7C914263
S315080025A010D0DA681570DA68597C5D680132013135
S315080025B0AA425974DA6003D902590120DA6038BD93
S315080025C0012038BD002038BD8C510008CC070020FA
S315080025D0012870B504460E4604D940F21A210E4861
S315080025E000F04CF904EB44040C4DE4002B19587C1C
S315080025F080B19A68127832709A68597C58680132A4
S315080026000139824259749A6003D92A5901209A607D
S3150800261070BD012070BD00BF8C510008CC0700209A
S31508002620F0B4144B144C1549651C04F14000144FC2
S3150800263003F1180201F140065A6158600022481C4D
S31508002640DE619D600126DD601D6040259A74DA62B0
S315080026505A7483F829203A601862586298610E7095
S3150800266083F82A601D7483F828502270F0BCFFF79F
S3150800267019B800BFCC07002080080020FC070020FE
S31508002680C80700200020FDF799BD00BF3F2970B597
S315080026900D46044621D8134E29463078FFF76EFFBB
S315080026A0012803D09D21104800F0E8F8ADB29DB18D
S315080026B0013DADB22544013C00F080F914F8011F34
S315080026C03078FFF75BFF01284FF0A601064801D0D6
S315080026D000F0D4F8AC42EFD170BD9921024800F061
S315080026E0CDF8D8E7800800208C510008F8B5194DB8
S315080026F00646FFF751FB2C7854B9174B174E187836
S315080027003146FFF765FF01281CD000242046F8BD96
S31508002710134C114B2178114F013139441878FFF7C2
S3150800272057FF0128F1D123783A780133DBB29A4270
S315080027302370EAD10446791C3046FFF76BFC002368
S315080027402B70E3E73378002BDFD0054B28701C701D
S31508002750DCE700BFC4070020FC070020C4080020EF
S3150800276044090020F0B51D4F83B03C78012C04D9EC
S3150800277040F23A211A4800F081F81A4B04EB440457
S3150800278003EBC404667C3EB3402E174D28BF402693
S3150800279000240DF107013878FFF71AFF012804F124
S315080027A001040F4803D040F2491100F067F89DF87C
S315080027B00720E3B29E4205F8012FEAD8B6B23246A0
S315080027C04FF480710948FFF74FF801203146FFF7AB
S315080027D017F90120FFF7B6F803B0F0BD800800200E
S315080027E08C510008CC0700200309002004090020AA
S315080027F070B50F4C01202146FFF7A0F980B290B1C1
S31508002800451EADB20B4E2544013C14F8011F307825
S31508002810FFF7B4FE01284FF4B771074801D000F05E
S315080028202DF8AC42F1D10120BDE87040FFF79EB803
S3150800283040080020FC0700208C51000810B50A4B00
S315080028400A490B4A1B680C681068181800D110BD95
S3150800285008220849FFF778FE2046BDE81040042202
S315080028600549FFF771BE00BFE8F7FF1FECF7FF1F2A
S31508002870F0F7FF1F060000201600002008B500F03C
S315080028809DF8FCE710B500F095F8012806D000F091
S3150800289009F918B10B4C2378012B00D010BDFFF7AE
S315080028A045FE094B1B6803F5FA639842F6D30023E5
S315080028B0237000F0FFF80028F0D1BDE81040FFF7BC
S315080028C089BB00BF450900204809002008B5054B0B
S315080028D001221A70FFF72AFE034B1860BDE808406C
S315080028E0FFF7D0BF450900204809002008B5FFF7C3
S315080028F06FFB00F061F8FFF7F1FDFFF7DBFD00F075
S31508002900BBF800F013F8BDE80840FFF7DFBF00BFCB
S3150800291008B500F053F8FFF7FBFD00F0CDF900F01D
S3150800292011F8BDE80840FFF7ADBF00BF08B502F0D3
S3150800293089F9FFF775FE024B02221A7008BD00BF1F
S31508002940EE00002008B50748FFF7D0FE012800D0A2
S3150800295008BD054B02221A700248BDE8084002F07D
S315080029608FB900BF4C090020EE000020FFF78ABE91
S3150800297008B5074B1B78022B03D0BDE8084002F0C8
S3150800298077B9C9B2FFF782FEBDE8084002F070B910
S31508002990EE000020044B1B78032B9ABF034A32F83B
S315080029A013003F20704700BFEE000020B451000816
S315080029B0FFF7F0BF02F054B9FDF73CBCFDF73EBC8B
S315080029C00209092A034615D903F00F033732092BE2
S315080029D00A701FD8124A3033126808461A445278C9
S315080029E002F00302022A08BF203BDBB200224B702A
S315080029F08A7070470A483032006803F00F031044A3
S31508002A00407800F00300022808BF203AD2B2092B0A
S31508002A100A70DFD9373300224B708A700846704730
S31508002A20F000002070B4134B411E1D68441C0020A2
S31508002A3011F8013FEA18527802F00302022A08BF89
S31508002A40203BDBB2A3F13002D2B2162AA3F13A0632
S31508002A500DD8062E0BD9092A84BF373BDAB202EB0A
S31508002A6000108C4200F0FF00E2D170BC70470020D5
S31508002A7070BC7047F000002008B5074A00231846C6
S31508002A800649137001F024FC00B908BD77210448F3
S31508002A90BDE80840FFF7F2BECC090020D80900209F
S31508002AA0BC510008024B1878B0FA80F0400970470C
S31508002AB0CC09002010B5FFF77DFF012802D0054C90
S31508002AC023780BB1002010BDFDF7BAFB0128F9D118
S31508002AD0207010BDCC0900200F4A03781168CA1867
S31508002AE0527802F00302022A08BF203B532B01D07A
S31508002AF003207047437819444A785207F8D5312B92
S31508002B0006D0322B06D0332B14BF03200220704781
S31508002B100020704701207047F000002070B5064677
S31508002B200230FFF77FFF0546043684B23046FFF7CA
S31508002B3079FF013CA4B22844012CC5B206F102066D
S31508002B40F4D83046ED43FFF76DFFEDB2281AB0FA18
S31508002B5080F0400970BD00BF2DE9F04104461646D5
S31508002B600F46002949D0002847D02046FFF7B4FF72
S31508002B70032805463ED02046FFF7D0FF002800F080
S31508002B809480012D64D03ED3022D33D1A01CFFF7CB
S31508002B9049FF0546201DFFF745FF4FEA0068C7F8BD
S31508002BA00080A01DFFF73EFF08EB0048C7F800802D
S31508002BB004F10800FFF736FF08EB0028C7F8008085
S31508002BC004F10A00FFF72EFF053D404438602DB298
S31508002BD00C3466B1002D0ADD00272046FFF722FFD8
S31508002BE07B1CF0559FB2AF4204F10204F5DB284680
S31508002BF0BDE8F0810020BDE8F08140F231212D4882
S31508002C00FFF73CFEB1E7A01CFFF70CFF0546201DA9
S31508002C10FFF708FF4FEA0028C7F80080A01DFFF756
S31508002C2001FF033D404438602DB20834002EDED043
S31508002C30002DDCDD00272046FFF7F4FE7B1CF0554F
S31508002C409FB2AF4204F10204F5DB2846BDE8F081E5
S31508002C50A01CFFF7E7FE0546201DFFF7E3FE4FEA37
S31508002C600048C7F80080A01DFFF7DCFE08EB002827
S31508002C70C7F8008004F10800FFF7D4FE043D40447D
S31508002C8038602DB20A34002EB1D0002DAFDD0027F2
S31508002C902046FFF7C7FE7B1CF0559FB2AF4204F1F2
S31508002CA00204F5DB2846BDE8F0814FF0FF30BDE8A9
S31508002CB0F08100BFBC5100082DE9F041C64F3C78B1
S31508002CC03CB1012C00F01381022C00F08D80032CFE
S31508002CD001D0BDE8F081C14DC14E05F50D723046F3
S31508002CE04FF4807101F01AFF95F93A32002BC0F2C1
S31508002CF03C81002855D006F5807206F5C07130462D
S31508002D00FFF72AFFB0F1FF3F804600F04181002817
S31508002D1047DDB448FDF7EAFA4346B349B34AA2FB8E
S31508002D200303DB0801F10101F9D14446AF480B70F2
S31508002D30A0FB0423DB0803EB8302A4EB4202303238
S31508002D4001F8012D1C46002BF2D1A748FDF7CEFA53
S31508002D50A748FDF7CBFAA44996F88301FFF730FE9A
S31508002D60A44996F88201FFF72BFEA34996F881013C
S31508002D70FFF726FEA14996F88001FFF721FE9A483B
S31508002D80FDF7B4FA9E48FDF7B1FA4146D6F8800138
S31508002D909C4AFFF791FB002800F0DB809A48FDF774
S31508002DA0A5FAD5F83C22D5F840329A4291D19748EF
S31508002DB0FDF79CFAFFF788FB0446002800F0FA8026
S31508002DC09148FDF793FA9248FDF790FA914801F079
S31508002DD04BFD9148FDF78AFA00233B70FDF766FA2A
S31508002DE0BDE8F041FFF7F6B87C4D7D4E05F50D724E
S31508002DF030464FF4807101F091FE95F93A32002B76
S31508002E00C0F2C18098B1002206F5C0713046FFF7BE
S31508002E10A3FE431C00F0DA80002808DD7F4C6368B7
S31508002E20002B40F08D80D6F8803160602360D5F89D
S31508002E303C22D5F840329A427FF44BAF00217548C0
S31508002E4001F01AFD002840F0A8806F48734CFDF782
S31508002E504DFA7348FDF74AFA656863492B46634A93
S31508002E60A2FB0303DB0801F10101F9D15F480B70EE
S31508002E70A0FB0523DB0803EB8302A5EB42023032F5
S31508002E8001F8012D1D46002BF2D15748FDF72EFA01
S31508002E906448FDF72BFA26685349300EFFF790FD74
S31508002EA05449C6F30740FFF78BFD5349C6F307207D
S31508002EB0FFF786FD5149F0B2FFF782FD4A48FDF754
S31508002EC015FA4F48FDF712FA94E80300FFF7F6FAE9
S31508002ED0002840F0B7805448FDF708FA0520FDF7AA
S31508002EE0FBF94C4801F0C0FC3D70BDE8F081FDF7E8
S31508002EF0C9F94E48FDF7FAF94D48FDF7F7F9FDF718
S31508002F00BDF922460146434801F0F2F9054638B1B3
S31508002F104548FDF7EBF92046BDE8F041FDF7DCB979
S31508002F203948FDF7E3F94348FDF7E0F94248FDF76C
S31508002F30DDF93A4B02221D605D603A70BDE8F0810A
S31508002F40D6F88021216818448A4238BF226060601A
S31508002F506DE73548FDF7CAF90620FDF7BDF92D4896
S31508002F6001F082FC3C70BDE8F0813448FDF7BEF9FB
S31508002F700220FDF7B1F905F50D7001F075FC002387
S31508002F803B70BDE8F0812848FDF7B0F92046F0E728
S31508002F902B48FDF7ABF92046EBE72348FDF7A6F9E2
S31508002FA00420FDF799F91B4801F05EFC00233B70ED
S31508002FB0BDE8F0811C48FDF799F90720FDF78CF963
S31508002FC0144801F051FC3C70BDE8F0811648FDF745
S31508002FD08DF90320CDE700BFCC090020D8090020D1
S31508002FE0300E0020F85200088C090020CDCCCCCC3D
S31508002FF0085300088E090020900900209209002035
S3150800300038530008300F00202C52000820530008BF
S315080030103C5300080C0C002054530008D00900202B
S31508003020885200089452000824520008D851000813
S31508003030FC5100083452000858520008B0520008E3
S31508003040D45200080348FDF751F903233B70BDE845
S31508003050F08100BF2C52000830B108B503680BB1E7
S315080030601A781AB9092008BD092070478288D988B4
S315080030709142F7D15878FDF7D1FB10F0010F14BF34
S315080030800320002008BD00BF2DE9F041036901F1C6
S315080030900902002B4DD0466901F1110496F80CE09F
S315080030A0751E0EF00807FFB20DE0A3F1410C37B10B
S315080030B0BCF1190F03F1200C01D85FFA8CF302F862
S315080030C0013BA2420AD015F8013F202B5DD0052B03
S315080030D0EBD1E52302F8013BA242F4D1337A22462A
S315080030E0202B18D00EF0100E2E235FFA8EF5013421
S315080030F002F8043BF71D17F8013F202BA3F1410EF8
S3150800310049D025B1BEF1190F9CBF2033DBB204F8B4
S31508003110013B9442EFD1F37A0B72F3690B60747E2C
S31508003120337E43EA04238B80F47DB37D43EA04238C
S31508003130CB80002414708E6936B1CB6923B103693C
S3150800314023B9002400233355BDE8F0814FF6FF73F9
S31508003150028C9A42F5D0C76938880028F1D00D4606
S3150800316006F1FF380BE0EB69013BA34204F10104C9
S31508003170E7D908F8010F37F814000028E2D0002133
S3150800318001F026FD0028EED1DBE71446337A224605
S31508003190202BA7D1BFE72246BDE700BF10B50446DE
S315080031A00A46407804F134010123FDF741FB08B1D2
S315080031B0032010BD4AF6552294F8331294F8323299
S315080031C043EA0123934201D0022010BDD4F86A30A5
S315080031D0064A23F07F439342F7D0D4F8863023F08B
S315080031E07F43981A18BF012010BD00BF46415400FE
S315080031F0F8B504682378303B092B02D865783A2D50
S3150800320014D000230B60904B1D6805B30D602B7816
S3150800321014469BB16878FDF701FBC7070ED4ECB1DD
S3150800322000F0040303F0FF00B3B9F8BD023400252B
S3150800323004600D60002BE6D00B20F8BD0020287036
S315080032406870FDF783F9C60703D50320F8BD0C207F
S31508003250F8BD2CB1410703D50A20F8BD2046F8BDB4
S3150800326000212846FFF79AFF012806D000240328E4
S3150800327000F0988060B10D20F8BD95F8F631002B66
S31508003280F9D0D5F8FA4128462146FFF787FFEEE739
S3150800329095F8402095F83F3043EA0223B3F5007FBE
S315080032A0E9D195F84B1095F84A3095F8447053EAE9
S315080032B0012314BF1946A96D7B1E012BE961EF7026
S315080032C0D9D895F84130AB70002BD4D05A1E1A4283
S315080032D0D1D195F8452095F8466042EA0626320788
S315080032E02E81C8D195F8480095F8472095F843E00F
S315080032F052EA002295F8420008BF6A6D50EA0E208D
S31508003300B9D001FB07F700EB161EBE447245B2D3CF
S31508003310CEEB0202B2FBF3F3002BACD040F6F5720B
S31508003320934271D94FF6F572934252D9023320442B
S3150800333004EB0E02AB616862EA622C62002E9AD137
S315080033409B002A6E03F2FF13B1EB532FAA6292D3A6
S3150800335095F8643095F865204FF0FF3143EA02226C
S3150800336022442961EE606E716A61012305F1340118
S315080033706878FDF75DFA48B94AF6552295F833128A
S3150800338095F8323243EA012393420DD003232F499D
S315080033902B700A880020531C9BB20B80EB80286395
S315080033A02871F8BD0120F8BD294B6A6B9A42EDD108
S315080033B003F1FF5303F50053D5F8182220339A4238
S315080033C0E4D1D5F81C32D5F820222B61EA60032314
S315080033D0DDE70233204404EB0E02AB616862EA6261
S315080033E02C62002E3FF447AF5B0003F2FF1338440C
S315080033F0B1EB532FA862FFF43EAF00234FF0FF3224
S31508003400EB602A610223C2E70233204404EB0E0272
S31508003410AB616862EA622C62002E3FF42CAF03F0BF
S31508003420010202F2FF1203EB430302EB5303384493
S31508003430B1EB532FA862FFF41EAF00234FF0FF3203
S31508003440EB602A610123A2E7B8110020B41100201D
S3150800345052526141F8B5056B00F1340704462A4615
S31508003460394640780123FDF737FAC0B9626A2071F8
S31508003470954212D3E3691A4495420ED2E678012E94
S3150800348001D80AE0E3691D44013E2A46012339466C
S315080034906078FDF721FA012EF4D10020F8BD01204D
S315080034A0F8BD00BFF8B5037905465BB92B78032B41
S315080034B00DD0002268781146FDF776FA003018BF5D
S315080034C00120F8BDFFF7C6FF0028EFD0F8BD6B79DD
S315080034D0002BEED005F134010B46002210462A6374
S315080034E005F50D7203F8010B93424FF00004F9D16C
S315080034F02A69EB6810124FEA124E170E1E1285F84B
S315080035001C2285F81D021A0E180C85F81EE285F88D
S315080035101F724FF0550E85F8203285F82162722306
S31508003520522685F8220285F8232261204122AA27FD
S3150800353085F8360085F81B0285F8372085F81A22A3
S3150800354085F8183285F8193285F832E285F833722B
S3150800355085F8346085F8356001236A696878FDF76F
S31508003560BBF96C71A5E700BF38B5036B8B4213D066
S31508003570037904460D464BB901232A4604F1340162
S315080035806078FDF755F928B9256338BDFFF762FF5E
S315080035900028F1D0012038BD002038BDF8B50378E1
S315080035A00546022B0C4646D0032B28D0012B02D009
S315080035B04FF0FF30F8BD416A04EB540601EB562183
S315080035C0FFF7D2FF0028F3D1696AC6F30803771C10
S315080035D02B4401EB5721284693F83460FFF7C4FFC4
S315080035E00028E5D1C7F308073D4495F83400E307FA
S315080035F046EA00204CBF0009C0F30B00F8BD416A3B
S3150800360001EBD411FFF7B0FF0028D1D1A30003F4D2
S31508003610FE742B1993F8362093F8371093F8350073
S31508003620120493F8343042EA016242EA0020184351
S3150800363020F07040F8BD416A01EB1421FFF794FFB2
S315080036400028B5D1640004F4FF742B1993F83500EB
S3150800365093F8343043EA0020F8BD00BF70B50D4634
S315080036608168C580012904D00446006883699942A7
S3150800367001D3022070BDB1B90378032B10D0002303
S31508003680E3600389AB42F4D9836A03EB151323611C
S3150800369005F00F05343000EB45106061002070BD61
S315080036A0816A0029EBD086783601B5420FD215E03B
S315080036B0FFF774FFAD1B431C0146ADB21DD00128B0
S315080036C0D7D9206883698B42D3D9AE4206D8012957
S315080036D0CFD983699942EBD3022070BDE160836933
S315080036E00239023B99423BBF8378C26A002101FB3B
S315080036F0032101EB15112161CAE7012070BD00BF46
S315080037002DE9F84390F800900446B9F1020F0D46EA
S31508003710174652D0B9F1030F2DD0B9F1010F05D0D4
S315080037200226012323713046BDE8F883416A05EB7A
S31508003730550801EB5821FFF717FF06460028F0D178
S31508003740C8F30803EA0723444DD593F8342008F153
S31508003750010802F00F0242EA071283F83420616A70
S3150800376084F8049001EB58212046FFF7FDFE002857
S3150800377054D00646D5E7416A01EBD511FFF7F4FEAA
S3150800378006460028CDD1AD0005F4FE75631993F8F9
S315080037903720120602F0704217433812390C3A0ED7
S315080037A083F8350083F8347083F8361083F83720A9
S315080037B0012323713046BDE8F883416A01EB1521E0
S315080037C0FFF7D2FE06460028ABD16D0005F4FF755B
S315080037D062193B1282F83530012382F8347023715E
S315080037E03046BDE8F88383F83470616A08F1010849
S315080037F084F8049001EB58212046FFF7B5FE00280F
S31508003800B7D1C8F30808A04498F83420C7F30327AB
S3150800381022F00F02174388F8347082E7C8F30808C5
S31508003820A044C7F30717F6E7F8B505460F46E9B902
S31508003830C668836946BB0126344610E0012E27D99F
S31508003840022B11D9022421462846FFF7A7FE08B302
S31508003850411C41D0012807D0A64219D0AB690134D2
S315080038609C42EBD2012CEED80120F8BD0129FBD9E8
S3150800387083699942F8D2FFF791FE0128F4D9AB691A
S315080038808342F2D83E46D7E79E4228BF0126D3E7B1
S315080038900020F8BDAB69A342E6D96FF07042214615
S315080038A02846FFF72DFFA8B957B1012FDCD9AB6918
S315080038B09F42D9D2394622462846FFF721FF48B902
S315080038C02B69EC605A1C0AD0013B01222B616A71F4
S315080038D02046F8BD0128C7D14FF0FF30F8BD204675
S315080038E0F8BD00BF2DE9F047C4880134A4B214B965
S315080038F00420BDE8F0870369002BF9D014F00F0700
S315080039000E46054608D00068343000EB471068615B
S31508003910EC800020BDE8F087C168013303610068C8
S3150800392061B18378013B13EA1413EDD1012902D959
S315080039308369994206D30220BDE8F0870389A3422A
S31508003940D6D9E1E7FFF72AFE01288046F3D9B0F178
S31508003950FF3F1CD02868836943450ED9A8F10206A3
S31508003960C5F80C808369023B9E423BBF8378C26AD6
S31508003970002606FB03262E61C6E7002EB8D0E968A6
S31508003980FFF752FF804628B90720BDE8F0870120D7
S31508003990BDE8F0870128CED0B0F1FF3FF7D0286800
S315080039A00379002B31D100F13403002200F50D70A4
S315080039B003F8012B9842FBD12B68A8F102069A69F5
S315080039C04FF00009023A96423BBF9A78D96A00221C
S315080039D006FB02124FF0010A1A6304E0036B09F1B1
S315080039E00109013303632B685FFA89F19A788A42E1
S315080039F011D983F804A028680379002BEED0FFF7C5
S31508003A0029FD0028C3D12868E8E7FFF723FD002829
S31508003A10BDD12868C7E71A6B521A1A6328689FE748
S31508003A20F8B54FF6FF73C588018C0446994208BF5E
S31508003A302946FFF713FEB8B9E52701260BE06369A7
S31508003A401F7023681E71E388AB420DD201462046DB
S31508003A50FFF748FF28B921692068FFF785FD002888
S31508003A60EDD0042808BF0220F8BD00BF2DE9F04FAD
S31508003A70FF2585B007462C4608E00F2940D0FF24CD
S31508003A8000213846FFF72EFF002836D139693868F5
S31508003A90FFF76AFD88BB7E693378002B78D0F27A07
S31508003AA0E52B02F03F01EAD01207E6D40F2927D00A
S31508003AB08CB91A463046234606F10A0401E010F886
S31508003AC0012FD90141EA53031344844203F0FF034B
S31508003AD0F5D1AB4210D04FF6FF72BB693A84DA7A59
S31508003AE0D207CCD403F10B0016F8011B13F8012BEF
S31508003AF09142C4D18342F7D1002005B0BDE8F08FCA
S31508003B00FA69002ABCD058063ED5F988757B03F0B9
S31508003B10BF04398496F80DA0AA45B0D13378DFF8EA
S31508003B20949023F04003013B012103EB430B084625
S31508003B304FF6FF7803EB8B0B09F10C0505E04345BF
S31508003B4031D14D4528D019F8011F731893F801E0B3
S31508003B50735C43EA0E230028F1D01846019201F05F
S31508003B6059F80BF10103BBF1FE0F039002931AD823
S31508003B70019A32F81B0001F04DF80399814212D1DF
S31508003B80029B019A9B46DCE7A3427FF478AFC1E724
S31508003B90042005B0BDE8F08F3378590606D528B15C
S31508003BA032F81B3013B15546FF2469E7631EDCB2B1
S31508003BB0554665E714540008F8B504460D4601272E
S31508003BC0A3699D4220D2012D0CD929462046FFF72C
S31508003BD0E5FC0646C0B1012804D0411C16D0A369ED
S31508003BE09D4201D30220F8BD294600222046FFF750
S31508003BF087FD60B9236935465A1CE1D00133236134
S31508003C00A36967719D42DED30020F8BD0120F8BD87
S31508003C102DE9F047FF2504462E46042006E0FF2638
S31508003C2000212046FFF75EFE00284ED121690029B3
S31508003C304FD02068FFF798FC002846D162691378B0
S31508003C40002B41D0E52BEAD02E2BE8D0D17A01F013
S31508003C503F010829E3D00F294CD1590631D5E1880F
S31508003C60557B03F0BF06218492F80DE0AE45D6D108
S31508003C7013782C4803F03F03013B012103EB43056E
S31508003C808C464FF6FF7AD4F81C9003EB850500F1B5
S31508003C900C0809E0FE2D11D89C4629F81530013587
S31508003CA080451BD010F8011F53185F78535C43EA10
S31508003CB00723BCF1000FEDD15345F1D07546FF2619
S31508003CC0AEE7B342ABD1CFE7042000232361BDE8BA
S31508003CD0F0870028F9D10020BDE8F08713785B0645
S31508003CE004D5FE2DEAD8002329F81530013EF6B290
S31508003CF0754695E78EB911461A4601F10A0033460C
S31508003D0001E011F8012FDE0146EA53031344884205
S31508003D1003F0FF03F5D1AB42DDD04FF6FF732384E2
S31508003D20D9E700BF145400082DE9F04F0B7883B08B
S31508003D302F2B0D46064600F035815C2B00F03281AC
S31508003D400024B46028781F2802D832E115F8010F3C
S31508003D502F28FBD05C28F9D080B21F28F76940F2DB
S31508003D60F6802F282ED05C282CD00121AA46A7F150
S31508003D700209012400F02CFF00B37F2809D8222865
S31508003D801CD09D4A01E0984218D012F8013F002B3A
S31508003D90F9D129F8020F1AF8010F631C1F2840F2FF
S31508003DA0D8802F2810D05C280ED0B3F5807F05D098
S31508003DB001211C4600F00CFF0028DED1062003B0C6
S31508003DC0BDE8F08F002401231D444FF0000A002CA3
S31508003DD0F4D007EB440232F8023D202B01D02E2BFB
S31508003DE002D1013CF7D1E9E7002327F81430B3697B
S31508003DF007EB440203F10B00202103F8011B834261
S31508003E00FBD1BB1E4FF0000901E009F1010933F8A7
S31508003E10020F2028F9D02E28F7D0B9F1000F01D0CB
S31508003E204AF0030A134633F8022D2E2A01D0013C24
S31508003E30F9D100239B464FF0080809F1010990B310
S31508003E40202820D02E281CD0434523D24C4500F0EC
S31508003E5084807F2800F28D802B2800F09980674A9D
S31508003E6002E0884200F0948012F8011F0029F8D178
S31508003E70A0F14101192900F2B4804BF0020BC0B23F
S31508003E8089E04C4504D04AF0030A37F81900D4E70C
S31508003E90434562D3B8F10B0F00F093804C455FD0D1
S31508003EA04AF0030A5CD2B3691978E52900F09280D2
S31508003EB0B8F1080F04BF4FEA8B0B5FFA8BFB0BF0C8
S31508003EC00C020C2A6BD00BF00301032967D01AF0F9
S31508003ED0020F0AD10BF0030BBBF1010F08BF4AF022
S31508003EE0100A042A08BF4AF0080A83F80BA0002122
S31508003EF03046FFF7B3FBB8B93046FFF7B7FDB369ED
S31508003F00DB7A98B959073FF55AAF7369DA7AD20658
S31508003F1012D53268D87E11789A7E032942EA0022A1
S31508003F200ED0B260287813E7B369DB7A04287FF4E9
S31508003F3046AF5C073FF543AF052003B0BDE8F08FF9
S31508003F40597D1B7D43EA012342EA0342E9E700243F
S31508003F5001231D444FF0040A39E7B8F10B0F30D09E
S31508003F604FEA8B0B5FFA8BFBA1464FF00B08082331
S31508003F708BE70021019300F02BFE019B70B3204ACA
S31508003F804AF0020A104410F8800C00287FF464AF47
S31508003F904AF0030A5F20B169C854013375E74AF04D
S31508003FA0020A94E700240135B46028781F283FF6F2
S31508003FB0CFAE21463046FFF751FB746103B0BDE82A
S31508003FC0F08FB3694AF0030A1A78E52A7FF477AFC7
S31508003FD04FF00B0805211970B36969E74AF0020A20
S31508003FE0D6E7A0F16101192997BF2038C0B2C0B23F
S31508003FF04BF0010BCFE700BF805300088C53000835
S315080040009453000870B4441E83B001F10B0611F8EE
S31508004010015BB14204F8015FF9D1052B0BD9118870
S3150800402000E02146DC0344EA530332F8024F0B440E
S315080040309BB2002CF5D102AD072203F00F0404F160
S315080040403001392988BF04F137011B0902F1FF3213
S3150800405005F8011DF1D102A97E24114401F8084C86
S31508004060F2B10178202908D0014603E011F8014F82
S31508004070202C02D001339A42F8D1184402A9072A03
S31508004080114498BF11F8081C03F101038CBF2021C5
S315080040900132072B00F8011BF0D903B070BC70473A
S315080040A01346EAE72DE9F04F876985B03B46044693
S315080040B0C66901AA07F10C0013F8011B834202F82E
S315080040C0011BF9D19DF80F30DA0723D50023FB72BF
S315080040D00125E36107E02046FFF7C8FC0135ADB2CC
S315080040E068B9642D78D001A938462B463246FFF7C1
S315080040F089FF00212046FFF7B1FA0028EBD00428F3
S3150800410002D005B0BDE8F08F9DF80F30FB729DF820
S315080041100F30E6619B074BD40125A84600212046AF
S31508004120FFF79CFA0028ECD1064605E0064620462D
S31508004130FFF7D8FB0028E4D121692068FFF714FAB5
S3150800414001210E440028DCD163691B78E52B01D0D8
S31508004150002BEBD1B542EAD108F1FF381FFA88F8EF
S31508004160B8F1000F3AD121692068FFF7FDF9002858
S31508004170C7D1636903F1200203F8010B9A42FBD108
S31508004180A369626903F10B00013A13F8011B834224
S3150800419002F8011FF9D1A3696169DB7A012203F0EC
S315080041A018030B73236800201A7105B0BDE8F08F59
S315080041B03388002BB0D0002301339BB236F8132086
S315080041C0002AF9D1404D193385FB0325DB17C3EBCC
S315080041D0A5051FFA85F8A1E7072092E7E18820469A
S315080041E0C8EB010189B2FFF739FA002889D183465D
S315080041F05B46A16901F10B0011F8012BDD0145EAC7
S3150800420053031344814203F0FF03F5D19B4623462B
S315080042104FF6FF7744469846D8F81010D8F80000AD
S31508004220FFF7A2F9014600287FF46BAF5FFA84FA1C
S315080042300AF1FF32034602EB420002EB80024FF01E
S315080042400F00D8F81460214DD8F81CC005F10C0EE3
S315080042503173B176F17686F80DB0F07201214FF020
S31508004260FF090EE03CF8123070187354190A002B37
S3150800427008BF3B46754502F1010241700AD015F8A0
S31508004280011FBB42EED17018754506F8019080F8FB
S315080042900190F4D1BB4202D03CF812300BB94AF077
S315080042A0400A86F800A0D8F8003001221A710021C9
S315080042B04046FFF717FB00287FF423AF013CA4B262
S315080042C0002CA9D144464EE74FECC44E14540008BE
S315080042D008B10B207047054B1A6802B1107009B176
S315080042E000220A7019600020704700BFB81100202C
S315080042F02DE9F0418EB0019130B3002305461446EE
S31508004300036005A902F01E0201A8FEF771FF10B1AD
S315080043100EB0BDE8F081514A02AB019905A80C928E
S315080043200B93FFF701FD04F01F070A9E80B9002EC4
S315080043304DD014F01C0F1CD0F37A13F0110F3BD19B
S31508004340600712D50820E3E709200EB0BDE8F08122
S3150800435014F01C0FDCD00428DAD105A8FFF7A2FE5A
S315080043600A9E0028D4D147F00807390731D4059B9F
S315080043700BE0F37ADA0621D4A00701D5D9071BD4B6
S315080043802207059B01D547F020071A6B2E62EA61C2
S31508004390AF711978F07EB27E032942EA00220FD067
S315080043A02A61F2690020EA602B60A860A861DB88B0
S315080043B0AB800EB0BDE8F0810720A9E70420A7E787
S315080043C0707D317D41EA002142EA0142E8E7062094
S315080043D09EE7FCF7F9FB0022040C010E4FEA202E9B
S315080043E0059B34747174B07386F80FE0F2723277F5
S315080043F07277B277F2771A78F47EB17E032A41EAA9
S3150800440004240FD000220121B276F2763275727535
S315080044101971002CB7D08C4202D99A69944208D3F4
S31508004420022075E7717D327D42EA012244EA0244A0
S31508004430E8E721461846D3F83080FFF7BDFB002889
S315080044407FF466AF0598013C4146C460FFF78CF8D7
S3150800445000287FF45DAF059B95E700BFB40F0020E9
S315080044602DE9F04F1E46002383B033600F46904671
S315080044700446FEF7F1FD28B9A3791D0605D4D80729
S3150800448007D4072003B0BDE8F08F022003B0BDE8CB
S31508004490F08FA268E568AD1A454528BF4546002D48
S315080044A000F0A980C2F3080304F1240904F5097889
S315080044B0002B41D120688378013B03EA522313F08D
S315080044C0FF034BD061698269A1F1020A023A92455B
S315080044D072D28178C26A01FB0A22002A6CD05FEA8E
S315080044E0552B02EB030A43D003EB0B02914238BF6C
S315080044F0C3EB010B5FFA8BF3407852463946FCF75B
S3150800450097F9A37900285ED15A0604D5A369CAEBA0
S31508004510030AD3455CD8A3684FEA4B2B5B44A360D8
S315080045203368B5EB0B055B445F44336063D0A26820
S31508004530C2F30803002BBDD0C3F5007BAB4528BFEB
S31508004540AB462344243303EB0B007A1E13F8011BF6
S31508004550984202F8011FF9D1A368DFE732BB226946
S31508004560012A29D9511C2DD0114620686261AAE773
S31508004570A269924514D0A3795B060AD5012340782F
S315080045804946FCF7A9F9A379E8B923F0400320685E
S31508004590A3714078012352464946FCF749F988B980
S315080045A0A368C4F818A0C3F30803C5E7616901291D
S315080045B002D98269914218D3A379022063F07F0356
S315080045C0A3715FE7A37963F07F030120A37159E71D
S315080045D007EB4A2A0AF1FF3204F1240313F8011BF8
S315080045E0434502F8011FF9D195E70193FEF7D6FF77
S315080045F0019B0246B4E7002044E700BF2DE9F84FC7
S315080046001F4600233B600C4616460546FEF724FD6A
S3150800461028B9AB79180604D4990705D40720BDE84C
S31508004620F88F0220BDE8F88FEA68D64209D3A96850
S3150800463043F02003914288BFE960AB710020BDE8D2
S31508004640F88F002EF3D005F12408AB68C3F30802EF
S31508004650002A6CD1286890F802B00BF1FF3B0BEAF0
S31508004660532B1BF0FF0B0DD1002B40F089802969D5
S31508004670002900F08D80012900F09C804A1C78D022
S3150800468028686961AB795B0666D46B698269A3F1B0
S31508004690020A023A924580F08D808278C36A02FB4C
S315080046A00A33002B00F086805FEA562903EB0B0AD3
S315080046B032D00BEB09039A4238BFCBEB020940789C
S315080046C05FFA89F352462146FCF706F9002850D1CD
S315080046D0AB69CAEB030399450FD904EB432303F5EA
S315080046E0007005F1230213F8011B834202F8011F2B
S315080046F0F9D1AB7923F04003AB714FEA4929AB688E
S315080047004C444B44AB603B68B6EB09064B443B60F4
S315080047109BD1EA68AB798AE7AB69AA689A4502D061
S31508004720EB689A423CD3C5F818A0C2F30802C2F552
S315080047300079B14528BFB1462A44234623324C4462
S3150800474013F8011B9C4202F8011FF9D1AA79AB683C
S3150800475042F04002AA71D4E701234078AA6941468B
S31508004760FCF7BAF8AB7928B923F040032868AB718F
S315080047708BE7AB7963F07F03AB710120BDE8F88F57
S315080047806969FFF751F8014600297FF474AFC0E75D
S31508004790FFF74AF80146286100297FF46CAFB8E7AD
S315080047A04078012352464146FCF742F80028E0D1FA
S315080047B0AA68B8E7AB79022063F07F03AB71BDE85E
S315080047C0F88F00BF70B50546FEF746FCD8B9AA793A
S315080047D002F0200303F0FF00ABB153060DD52A689B
S315080047E00123507805F12401AA69FCF775F8002819
S315080047F037D1AB7923F04003AB71E9692868FEF736
S31508004800B3FE044600B170BD2E6AF37A43F0200366
S31508004810F372EB683377EB681B127377EB89B37720
S31508004820EB7BF3772B691A0C11121812B3763275D3
S315080048307175F076FCF7C8F90112020C030EF175D2
S31508004840B075B474F47432767376AB792A6823F04B
S3150800485020030121AB7111712868BDE87040FEF78D
S3150800486021BE012070BD00BF10B50446FFF7AAFFA0
S3150800487000B9206010BD00BF70B50E460446FEF7AD
S31508004880EBFB002846D1A3791D0644D4E268B24260
S3150800489003D213F0020F08BF16460022A368A260CF
S315080048A0002E3AD0206885786D0243B1013B721E0E
S315080048B0B3FBF5F1B2FBF5F28A4280F081802169FB
S315080048C0002900F08380616149BB0D46A368C3F3E4
S315080048D00802002A00F08380A26995427FD0A37956
S315080048E05B065ED404F124062368314658782A46C6
S315080048F00123FBF79DFF00284DD1A368E268A56157
S315080049009A4206D2A279E36042F02003A3710020FE
S3150800491070BD002070BD022070BD304670BDAE422D
S3150800492068D92068A379761B9A0709D4012902D980
S3150800493082698A422BD863F07F03A371022070BD77
S31508004940FEF772FF0146002853D04A1C23D00129DE
S315080049504DD920688369994249D2A368B5422B4448
S31508004960A3606161DED33344C6F30805A360002D56
S31508004970ADD0206802398269023A914231D28278F2
S31508004980C56A01FB025161B301EB56259FE7FEF7A5
S3150800499005FE0146D9E7A37963F07F03A3710120D9
S315080049A070BD236804F12406587831460123FBF7C5
S315080049B093FFA3790028EFD123F04003A37193E76F
S315080049C06A421340A360F61A61697DE7FEF72CFF79
S315080049D00128014605D00130DDD0216173E7E26880
S315080049E08EE7A379022063F07F03A37170BDA379D4
S315080049F0A1E72E46A368B6E730B58FB001900D46FD
S31508004A00002205A901A8FEF7F3FB044610B12046CB
S31508004A100FB030BD0B4A02AB019905A80C920B9357
S31508004A20FFF782F904460028F1D10A9B33B105A89D
S31508004A302946FEF729FB20460FB030BD062420463E
S31508004A400FB030BDB40F002030B599B0019006A95B
S31508004A50012201A8FEF7CCFB08B119B030BD2E4AD9
S31508004A6003AB019906A80D920C93FFF75DF9002890
S31508004A70F3D10B9B002B4BD0DA7A12F0010F0CBF47
S31508004A8000200720069ADD7E1278997E032A41EADD
S31508004A9005252BD00028E0D1DB7ADB0618D5012DB9
S31508004AA022D906AC0DF13B030FA914F8012B8C4251
S31508004AB003F8012FF9D1022120461195FEF7CEFD04
S31508004AC00028CAD12046FFF7A3F818B30428C4D192
S31508004AD006A8FEF7A5FF0028BFD1ADB1012D03D961
S31508004AE006988369AB420AD80220B6E7597D1A7D33
S31508004AF042EA012245EA02450028AED1CCE729461A
S31508004B00FFF75AF80028A8D10698FEF7CBFCA4E7C9
S31508004B100620B7E70720A0E7B40F00202DE9F041EB
S31508004B2080461746054682B04E1E0024B4424FF012
S31508004B30010212DA01AB69463846FFF791FC019B80
S31508004B406A1C012B09D19DF800300D2BEED00A2BDB
S31508004B502B7004F101041546E8D1002C4FF0000330
S31508004B6014BF404618462B7002B0BDE8F08100BF5E
S31508004B7030B50A2883B004460D460FD001AB284647
S31508004B80012269468DF80040FFF738FD019B012B8D
S31508004B900CBF01204FF0FF3003B030BD0D20FFF7EA
S31508004BA0E7FFEBE7037883B170B50E460546441C6C
S31508004BB003E0601B14F8013B33B118463146FFF792
S31508004BC0D7FF431CF5D170BD70BD1846704700BFAE
S31508004BD07F2811D989B910B40D4AC72303E0802963
S31508004BE014D032F8023F98428CB201F10101F6D195
S31508004BF004F1800080B210BC7047FF2804D8044B2B
S31508004C00803833F810007047002070470020F2E71C
S31508004C100456000861280FD008496223002203E0E1
S31508004C20984205D031F8023F0132002BF8D170477F
S31508004C30034B33F8120070474120F8E72654000862
S31508004C4004570008054B00221A709A6483F842201C
S31508004C50A3F844209A705A70704700BFBC11002010
S31508004C60024B1878003018BF01207047BC1100208D
S31508004C70024B002283F84220704700BFBC11002077
S31508004C8070B50578FF2D41D0B44C2378012B00D0A0
S31508004C9070BDC93D0646352D00F24681DFE815F0A0
S31508004CA0FF0044014401700044014401780080007B
S31508004CB0A000AD00440144014401440144014401FB
S31508004CC044014401440144014401440144014401AE
S31508004CD0440144014401440144014401440144019E
S31508004CE0440144014401440144014401440144018E
S31508004CF044014401BC00D4003001170144014401B9
S31508004D0044011F014401E100E900F600FDF7CAFE6F
S31508004D10924CE8B9FE2110220223E1702271A4F810
S31508004D20443094F842308D4A012B09D0B2F8441029
S31508004D30012384F842308A48BDE87040FDF718BE62
S31508004D40FE2210230221E2702371A4F84410EFE733
S31508004D50002310220126637063712271E5702670A4
S31508004D60FDF726FEA071FDF715FEE071FDF712FEB0
S31508004D700823D84020726672A672A4F84430D0E799
S31508004D80FE2131220223E1702271A4F84430C8E7DB
S31508004D90FDF720F9FF220123E270A4F84430C0E7AA
S31508004DA0FDF706FE73780138984252DDFF2201238B
S31508004DB0E270A4F844307178684D002940F0C1804B
S31508004DC0FDF782FB0028DBD094F84220634B012ACA
S31508004DD0B6D0B3F9441000297FF75AAF89B2A7E7CE
S31508004DE04168A06C5D4DFDF769FB0028C8D0FF221D
S31508004DF00123EA70A5F8443093E70025FF23E37002
S31508004E0025716571FDF7D4FD0723A071E57125723B
S31508004E106572A4F8443084E7FF23E3704368A26C04
S31508004E203BB1D018002312F8011B0B448242DBB2B7
S31508004E30F9D1002201200821C4F8073020716271D7
S31508004E40A271A4F844106CE7FDF7B2FD7378984296
S31508004E5072DCFE2122220223E1702271A4F844307A
S31508004E605FE7FE2100220223E1702271A4F8443094
S31508004E7057E760780023FF2106226071E1702371ED
S31508004E80A371E3712372A4F844204AE70023FF21A3
S31508004E90012223706370E170A4F8442041E7A56CF1
S31508004EA0FDF786FD721C411E28462C4DFDF704FBB6
S31508004EB000283FF465AFFF23EB70FDF779FDAB6C77
S31508004EC0013803440122AB64A5F8442029E7FF23EF
S31508004ED0E37042680123A264A4F8443021E7214D17
S31508004EE00023FF2007210822A564E070237163715F
S31508004EF0A37123726372A372E171A4F8442010E7C8
S31508004F00FDF756FD72789042A3DDA16C1648FDF7B1
S31508004F1081F8FF23E3707378A26C1344A364737853
S31508004F200133A4F844304FE7FE2120220223E17022
S31508004F302271A4F84430F4E671680B48A1647278CB
S31508004F40E5E7B21CA86CFDF7B7FA00283FF418AFDE
S31508004F507378AA6C1344AB6436E700BFBC11002013
S31508004F60BF110020E4580008C011002008B5074BFF
S31508004F70044613B10021AFF30080054B1868836A15
S31508004F8003B19847204600F033F800BF0000000040
S31508004F90F05900080E4B70B51E460E4C0025E41A53
S31508004FA0A410A54204D056F8253098470135F8E7ED
S31508004FB000F020F8084B094C1E46E41AA4100025F8
S31508004FC0A54204D056F8253098470135F8E770BD54
S31508004FD054010020540100205401002058010020EB
S31508004FE003460244934202D003F8011BFAE77047CE
S31508004FF0FEE70000F8B500BFF8BC08BC9E4670473F
S31508005000F8B500BFF8BC08BC9E4670472F64656DAE
S315080050106F70726F675F6F6C696D6578696E6F5FC9
S3150800502073746D33322E7372656300002F626F6F6F
S31508005030746C6F672E747874000000002E2E5C6DF9
S3150800504061696E2E63000000120110010000004025
S31508005050501DAC60000101020301000004030904AD
S315080050602603570069006E005500530042002000D1
S31508005070420075006C006B00200044006500760055
S31508005080690063006500000009022000010100C0F4
S31508005090320904000002FF000004070581024000EF
S315080050A000070501024000001A034F007000650062
S315080050B06E0042004C005400200055007300650045
S315080050C0720000002C03570069006E00550053005B
S315080050D042002000420075006C006B002000490069
S315080050E06E0074006500720066006100630065006A
S315080050F0006000080020000003000000008000088F
S31508005100002000000400000000A0000800200000A5
S315080051100500000000C0000800200000060000008E
S3150800512000E0000800200000070000000000010859
S3150800513000200000080000000020010800200000F0
S315080051400900000000400108002000000A000000D5
S3150800515000600108002000000B0000000080010824
S31508005160002000000C00000000A00108002000003C
S315080051700D00000000C00108002000000E0000001D
S3150800518000E00108002000000F0000002E2E5C2E13
S315080051902E5C2E2E5C2E2E5C536F757263655C41F9
S315080051A0524D434D335F53544D333246315C75731C
S315080051B0622E6300000008003F0000002E2E5C2EC1
S315080051C02E5C2E2E5C2E2E5C536F757263655C66A4
S315080051D0696C652E630000004669726D77617265B9
S315080051E020757064617465207265717565737420C5
S315080051F064657465637465640A0D00004F70656EB6
S31508005200696E67206669726D776172652066696C7A
S315080052106520666F722072656164696E672E2E2E30
S31508005220000000004552524F520A0D004F4B0A0D1E
S31508005230000000005374617274696E6720746865B3
S315080052402070726F6772616D6D696E672073657124
S3150800525075656E63650A0D0050617273696E672025
S315080052606669726D776172652066696C6520746F10
S31508005270206F627461696E20657261736520736957
S315080052807A652E2E2E00000045726173696E6720BE
S31508005290000000002062797465732066726F6D20C5
S315080052A06D656D6F7279206174203078000000009A
S315080052B052656164696E67206C696E652066726FF7
S315080052C06D2066696C652E2E2E4552524F520A0D78
S315080052D000000000496E76616C6964206368656346
S315080052E06B73756D20666F756E642E2E2E45525241
S315080052F04F520A0D0000000050726F6772616D6DA3
S31508005300696E672000000000206279746573207456
S315080053106F206D656D6F727920617420307800009A
S3150800532057726974696E672070726F6772616D2053
S31508005330636865636B73756D2E2E2E00436C6F73F1
S31508005340696E67206669726D776172652066696C39
S31508005350650A0D004669726D77617265207570641D
S31508005360617465207375636365737366756C6C79B0
S3150800537020636F6D706C657465640A0D000000002B
S31508005380222A3A3C3E3F7C7F000000002B2C3B3D06
S315080053905B5D0000809A90418E418F804545454966
S315080053A049498E8F9092924F994F555559999A9B84
S315080053B09C9D9E9F41494F55A5A5A6A7A8A9AAABFE
S315080053C0AC21AEAFB0B1B2B3B4B5B6B7B8B9BABB23
S315080053D0BCBDBEBFC0C1C2C3C4C5C6C7C8C9CACB87
S315080053E0CCCDCECFD0D1D2D3D4D5D6D7D8D9DADB77
S315080053F0DCDDDEDFE0E1E2E3E4E5E6E7E8E9EAEB67
S31508005400ECEDEEEFF0F1F2F3F4F5F6F7F8F9FAFB56
S31508005410FCFDFEFF01030507090E10121416181CE1
S315080054201E000000610062006300640065006600FB
S315080054306700680069006A006B006C006D006E000A
S315080054406F007000710072007300740075007600BA
S315080054507700780079007A00A100A200A300A500D1
S31508005460AC00AF00E000E100E200E300E400E50084
S31508005470E600E700E800E900EA00EB00EC00ED00D2
S31508005480EE00EF00F000F100F200F300F400F50082
S31508005490F600F800F900FA00FB00FC00FD00FE002B
S315080054A0FF00010103010501070109010B010D01B7
S315080054B00F01110113011501170119011B011D0126
S315080054C01F01210123012501270129012B012D0196
S315080054D02F0131013301350137013A013C013E0103
S315080054E0400142014401460148014B014D014F016B
S315080054F0510153015501570159015B015D015F01D6
S31508005500610163016501670169016B016D016F0145
S3150800551071017301750177017A017C017E0192019F
S31508005520B103B203B303B403B503B603B703B803B1
S31508005530B903BA03BB03BC03BD03BE03BF03C00361
S31508005540C103C303C403C503C603C703C803C9030A
S31508005550CA033004310432043304340435043604EF
S315080055603704380439043A043B043C043D043E0439
S315080055703F044004410442044304440445044604E9
S315080055804704480449044A044B044C044D044E0499
S315080055904F04510452045304540455045604570442
S315080055A0580459045A045B045C045E045F047021C1
S315080055B07121722173217421752176217721782131
S315080055C079217A217B217C217D217E217F2141FF42
S315080055D042FF43FF44FF45FF46FF47FF48FF49FF99
S315080055E04AFF4BFF4CFF4DFF4EFF4FFF50FF51FF49
S315080055F052FF53FF54FF55FF56FF57FF58FF59FFF9
S315080056005AFF0000C700FC00E900E200E400E000E1
S31508005610E500E700EA00EB00E800EF00EE00EC002A
S31508005620C400C500C900E600C600F400F600F20092
S31508005630FB00F900FF00D600DC00A200A300A500CD
S31508005640A7209201E100ED00F300FA00F100D10075
S31508005650AA00BA00BF001023AC00BD00BC00A10020
S31508005660AB00BB00912592259325022524256125AB
S315080056706225562555256325512557255D255C2523
S315080056805B251025142534252C251C2500253C25AD
S315080056905E255F255A2554256925662560255025EA
S315080056A06C256725682564256525592558255225BD
S315080056B053256B256A2518250C25882584258C25D0
S315080056C090258025B103DF009303C003A303C3031A
S315080056D0B500C403A6039803A903B4031E22C60390
S315080056E0B50329226122B1006522642220232123E1
S315080056F0F7004822B0001922B7001A227F20B2000C
S31508005700A025A00041004200430044004500460091
S315080057104700480049004A004B004C004D004E0027
S315080057204F005000510052005300540055005600D7
S315080057305700580059005A002100E0FFE1FFE5FF35
S31508005740E2FFE3FFC000C100C200C300C400C500F9
S31508005750C600C700C800C900CA00CB00CC00CD00EF
S31508005760CE00CF00D000D100D200D300D400D5009F
S31508005770D600D800D900DA00DB00DC00DD00DE0048
S315080057807801000102010401060108010A010C0161
S315080057900E01100112011401160118011A011C014B
S315080057A01E01200122012401260128012A012C01BB
S315080057B02E01300132013401360139013B013D0128
S315080057C03F0141014301450147014A014C014E0190
S315080057D0500152015401560158015A015C015E01FB
S315080057E0600162016401660168016A016C016E016B
S315080057F0700172017401760179017B017D019101C5
S3150800580091039203930394039503960397039803CE
S3150800581099039A039B039C039D039E039F03A0037E
S31508005820A103A303A403A503A603A703A803A90327
S31508005830AA0310041104120413041404150416040C
S315080058401704180419041A041B041C041D041E0456
S315080058501F04200421042204230424042504260406
S315080058602704280429042A042B042C042D042E04B6
S315080058702F040104020403040404050406040704AF
S31508005880080409040A040B040C040E040F0460211E
S3150800589061216221632164216521662167216821CE
S315080058A069216A216B216C216D216E216F2121FFEF
S315080058B022FF23FF24FF25FF26FF27FF28FF29FFB6
S315080058C02AFF2BFF2CFF2DFF2EFF2FFF30FF31FF66
S315080058D032FF33FF34FF35FF36FF37FF38FF39FF16
S315080058E03AFF00004F70656E424C5400002020209D
S315080058F02020202020202828282828202020202072
S315080059002020202020202020202020202088101041
S31508005910101010101010101010101010100404049D
S31508005920040404040404041010101010101041415B
S315080059304141414101010101010101010101010149
S31508005940010101010101010110101010101042425D
S315080059504242424202020202020202020202020219
S3150800596002020202020202021010101020000000B9
S315080059700000000000000000000000000000000019
S315080059800000000000000000000000000000000009
S3150800599000000000000000000000000000000000F9
S315080059A000000000000000000000000000000000E9
S315080059B000000000000000000000000000000000D9
S315080059C000000000000000000000000000000000C9
S315080059D000000000000000000000000000000000B9
S315080059E00000000000000000000000000043000066
S30D080059F0F4000020000000008D
S30D080059F850A7FF7F0100000023
S31508005A00010000001C03530045005200310032001B
S31508005A1033003400350036003700380039003000CE
S31508005A207D1D0008A1160008A1160008A116000889
S31508005A30A1160008A1160008A1160008811D000875
S31508005A40A1160008A1160008A1160008A11600084C
S31508005A50A1160008A11600088850000820000000BA
S31508005A60891E0008AD1E00089D1F0008311E00088B
S31508005A70351E0008751E0008791E0008591F000803
S31508005A80651F0008711F00080000000040000000A4
S31508005A90A11600080D1E0008A1160008A116000888
S31508005AA0A1160008A1160008A1160008A1160008EC
S31508005AB0251E00089A5000080900000048500008F2
S31508005AC0120000005C50000804000000A8500008FE
S31508005AD01A0000006050000826000000040000209C
S31508005AE01C000000C45000082C000000030104003C
S31508005AF0EC5800080000000000000000000000004C
S31508005B000000000000000000000000000000000087
S31508005B1000000000ED590008000000000000000029
S31508005B200000000000000000000000000000000067
S31508005B300000000000000000000000000000000057
S31508005B400000000000000000000000000000000047
S31108005B500000000011010008ED0000082C
S70508000000F2
